:0C0000001F308A005C2F00001028080050
:10002000FF00030E8301A1000A08A0008A01040852
:10003000A2007708A3007808A4007908A5007A0830
:10004000A600831383128C308400801E29288C1A0A
:100050003A28220884002308F7002408F80025081D
:10006000F9002608FA0020088A00210E8300FF0EFE
:100070007F0E09008A110A123D288C1E3D2818089F
:10008000A7001A08F800A71C4728181218167808A5
:100090008316B90083120C1E4B2899008C128A110A
:1000A0000A1229280D050D0523104226EF30E432EF
:1000B0007210381C3710A82129103218B119A02548
:1000C000C125CC060A002310D232F332723B6532CE
:1000D0003A102526F5060A0023104626C129C82F06
:1000E0004529C129C52FD324DA223A102526F50641
:1000F0000A0023104626C129C82F5729492AC52F8F
:10010000D324DA223A102526F5060A002310C23736
:100110006F3A2026EF30E4327210D432733A201F47
:100120003E1F0D05231000015F08E1005E08E0009E
:100130006108FA006008840083137A188317800826
:100140000319A628E00A0319E10A98285E0860024C
:10015000F7006108FA005F08031C5F0FFA027708D6
:10016000F8000800831603178C170C140000000019
:1001700083120C087F390319F8280313DE000317D4
:100180000D080313DF0003170F080313E0005E08D8
:100190000C1EC82899005F0803178D000313600820
:1001A00003178F0083168C170C14000000008312B5
:1001B0000C0D0E0D7F390319F8280313DE00031709
:1001C0000D080313DF0003170F080313E0005E0898
:1001D0000C1EE82899005F0803178D0003136008C0
:1001E00003178F008D0A03198F0A0313B228031710
:1001F00003130800831603178C170C14000000006B
:1002000003182A2983120C087F390313AD00031742
:100210000D080313AE0003170F080313AF002D08DA
:100220000C1E102999002E0803178D0003132F08A8
:1002300003178F0083168C170C1400000000831224
:100240000313AC0B24292729831603172A294A29CB
:100250008316031783120C0D0E0D7F390313AD00A7
:1002600003170D080313AE0003170F080313AF00A5
:100270002D080C1E392999002E0803178D00031331
:100280002F0803178F008D0A03198F0A0310031319
:10029000AC0BFA280800B4010408B3003410831B27
:1002A00034142D0EF038AF00AF07E23EB000323EFE
:1002B000B2002D080F39B007B007B207E93EB10010
:1002C000B107B1072C0E0F39B107B207B10DB20D4E
:1002D000B209B20D2C080F39B207AF0D0730AE00CE
:1002E0000A30B207B103031C7129B107B003031C24
:1002F0007529B007AF03031C7929AF07AE03031CB0
:100300007D292E308400831307303305331384078F
:1003100032300402031933170008F700031D98292F
:10032000331B9829331AA029B319982920309B2907
:10033000B31533123030F70777080C1E9D2999004A
:10034000840A331F882908003008F8012F02031897
:10035000AC292F08F700B829F7010830B100AF0D1C
:10036000F70D300877020318F700F80DB10BAF292D
:100370000800AB012708AB002430AC004930AD00C9
:100380006430AE003A30AF002030B0006230B100CF
:100390006C30B2006F30B3006130B4006430B5002F
:1003A0006530B6007230B7002E30B8006330B90047
:1003B0002030BA003230BB003830BC003130BD00D4
:1003C0003230BE002030BF003230C0003030C100BB
:1003D0003130C2003330C3002D30C4003030C5008E
:1003E0003330C6002D30C7003130C8003030C9006E
:1003F0002030CA003030CB003830CC003A30CD004D
:100400003030CE00CF003A30D0003230D10033301F
:10041000D2005A30D3002030D4006B30D500613088
:10042000D6006B30D7006C30D8002030D900243093
:10043000DA00DB01DF012C30DE009420013078028D
:100440002C3E840083130008243C031D312ADF0165
:100450002C30DE009420013078022C3E840083137F
:100460008001523003178D0000308F000313B2203B
:1004700023300C1E392A9900303084008313800801
:100480000319552ADF010408DE005F10831B5F1487
:1004900000080C1E492A99005E08840083135F1827
:1004A0008317840A0319850A3F2A0D300C1E562A29
:1004B00099000A300C1E5A2A9900633003178D00E8
:1004C00000308F0003100C300313AC00FA20103002
:1004D00084000330AD001030AC004B210D300C1EF9
:1004E0006F2A99000A300C1E732A99006C3003178A
:1004F0008D0000308F00031014300313AC00FA207D
:1005000010308400AD012030AC004B210D300C1EAA
:10051000872A99000A300C1E8B2A9900793003171C
:100520008D0000308F00031014300313AC00FA204C
:1005300010308400AD01AC004B210D300C1E9E2A02
:1005400099000A300C1EA22A9900863003178D00EC
:1005500000308F000313B22083168C16C030831234
:100560008B042B08AB0AAC002C08AD001B30AE008E
:100570002D08AF006430B000A4217708AD007808E2
:100580003030031DCA2AAE1CD22AAE19D22A2E1A26
:100590002030CD2AAE112E122E14F80778080C1E2A
:1005A000CF2A99002D08AF000A30B000A4217708A7
:1005B000AD0078083030031DE32AAE19E82A2E1C5E
:1005C000E82A2E1A2030F80778080C1EE52A990030
:1005D0003030AD072D080C1EEB2A99007C300C1E24
:1005E000EF2A99006430AC002C308400831300089B
:1005F0000319072B0230F800F701F70BFD2AF80B5F
:10060000FC2A9730F700F70B032B800BFA2AB12A4C
:060610008A150A16F32C06
:0C39E0000A128A11B9290A168A1508007B
:103A00008C1E002D1808A7001A08F800A71C0A2D04
:103A10001812181608008316B10803191F2D453017
:103A200083120C1E112D9900303083163207B3001B
:103A300083120C1E192D99008A0100288316831207
:103A400008008316B601B7013708013C031C552D49
:103A50003508FA003408840083137A1883170008A5
:103A6000403C0318422D360EB800F030B80534083B
:103A7000840083133518831700083807BF3E0A3EB9
:103A8000B6004F2D360EB800F030B805340884006B
:103A900083133518831700083807D03EB60037085F
:103AA000B70AB40A0319B50A242D3608F8008312A0
:103AB00008000B08F8008B138316031755308D0090
:103AC000AA308D008C14000000008C18652D0C119C
:103AD0007808831203138B040800831603178C17CE
:103AE00083120D08033903198A2DF9000D08FC39DA
:103AF0008D0083160C1483128D00000000008316C5
:103B00000C1583120313592503178D0A03198F0A05
:103B1000F90B7D2D831603133008F9000310F90CFF
:103B20000F30831203170D05031DA02D83160C16ED
:103B30000C15831203135925831603170C128312D5
:103B400000088C00840A00088E00840A83160C1575
:103B500083120313592503178D0A03198F0AF90BD2
:103B6000B22DB52D83160313902D0D0807390319B7
:103B7000C92D043CF900FF308C008E0083160C1513
:103B800083120313592503178D0A03198F0AF90BA2
:103B9000BB2D03130800E001DF010B138B138B1BFC
:103BA000CE2D21300C1ED22D99008C1AD92D6400F7
:103BB000D52D0D300C1EDA2D99000A300C1EDE2D8D
:103BC0009900002578083A3C0319E82D6400E12D9E
:103BD0003A300C1EE92D9900AB012C302B078400E4
:103BE0008313EC010408EB006C10831B6C1400259C
:103BF0006B08840083136C188317780880002C30BE
:103C00002B07840083130008E90069080C1E062EA8
:103C100099002B08AB0A2C3E8400831300080D3C4E
:103C20000319162E2B082D3C0318ED2D2B082E3CC6
:103C300003191C2E00301D2E0130E9008316B1003F
:103C40000130B20083120B25AB036400DA01E801F6
:103C50002B0868020318402E2C306807E900EA019F
:103C60000318EA0A6A088316B500831269088316E6
:103C7000B400831221257808DA070230E807282EDD
:103C8000DA08031D452E0030462E0130E900831668
:103C9000B1000230B20083120B258316B5012E301D
:103CA000B400831221257808E9008316B50130306D
:103CB000B400831221256908DE007808DD00831630
:103CC000B5013230B400831221257808DC00831658
:103CD000B5012C30B400831221257808DB005B0885
:103CE000103C031C752E0030762E0130E90083163F
:103CF000B1000330B20083120B255D08E1005E08BD
:103D0000E2000310E20CE10C5C0B8C2E23300C1E45
:103D1000872E99008A010028DC08031D912E0030AF
:103D2000922E0130E9008316B1000430B2008312F4
:103D30000B25E801E601E5016208E4006108E30003
:103D40006808073C031CD02E0310680DA03E8400B9
:103D500083136608FA006508F9006408F800630830
:103D6000F7000130E3070318E40A0319E50A031911
:103D7000E60A7A08EE00770803178D000313780827
:103D800003178F0083168C170C1400000000831299
:103D90000C088000840A0E0880000313E80AA02E95
:103DA0000830E800E70102302B0268020318FC2EFD
:103DB0006708E70AA03EF800FA010318FA0A780833
:103DC000E9007A08EA002C306807EB00EC010318E0
:103DD000EC0A6C088316B50083126B088316B400D6
:103DE000831221256908840083136A1883177808D1
:103DF00080000230E807D32EE108031D1B2FE208E4
:103E0000031D1B2F1C30E200F030E1006208031795
:103E10008F000313610803178D00A0308400831303
:103E2000103083160313B00083126D2525300C1E4D
:103E3000172F9900452FE208031D222F6108073C28
:103E40000318412F62081C3C031C412F031D2C2F1B
:103E50006108E03C031C412F620803178F00031325
:103E6000610803178D00A03084008313103083167F
:103E70000313B00083126D2524300C1E3D2F9900D2
:103E8000452F2E300C1E422F99000D300C1E462F50
:103E900099000A300C1E4A2F99006400E12D080099
:103EA000AC01AB012B0F572F2C0F572F5B2FAB0AF9
:103EB0000319AC0A522F0800840183131F308305B5
:103EC000713083168F000F08031787110C3003130E
:103ED0009900A2309800903083129800831603173F
:103EE00087110C3003139900A23098009030831290
:103EF0009800831603170908C039890003131F129D
:103F00009F120030031788008312870188018901FE
:103F10000313A701A801A9010B138B138B1B8D2F72
:103F20000930031785000F30F7000313810181303A
:103F3000840083130008F03907388000640000080B
:103F4000F739F719F0397704800083160317090849
:103F5000C039890003131F129F1200300317880015
:103F6000831203131F1083160108C7390838810014
:103F7000831290010030F800920000308316920006
:103F800083120317870188018901831603139701A0
:103F900071308F000F088312AA012A0FD02FF42F3F
:103FA0008C1EE42F00257808753C031DE32F2A3072
:103FB0000C1ED82F990000257808663C031DE22FBF
:103FC0006400CB25E42FF42F75300C1EE52F9900EB
:103FD00066300C1EE92F99003F300C1EED2F990022
:103FE00050276400AA0ACD2F64001C308A00F030EC
:043FF00082006300E8
:04400E00FD2CFF3F47
:00000001FF
